:020000040000FA
:04000000CF303A289B
:08000800A000030EA100831209
:1000100005191028831601178312B23081002B288E
:1000200083160113831203140B190310A80DA90DD5
:10003000AA0DAB0DAC0DAC16FF302C02031D2B2806
:10004000FA302B02031D2B2831152A08AF0029088E
:10005000AE002808AD008B100B11210E8300A00EFE
:04006000200E090065
:0C007400203084008001840A80300402E7
:10008000031C3C281230B000FA2183160C30850581
:1000900087018312850187010730990000309A009B
:1000A000103083168E008312603083168F00831207
:1000B0000030831691009F008312C83083168100A0
:1000C000831231309000003083168C008312103080
:1000D0008B00831600309B001C141A088312BC008E
:1000E000851D1A23831610309B001C141A088312D6
:1000F000BD00831630309B001C141A088312DE00EA
:10010000FD2281018E018F010B118B100B108C01D0
:100110008B17982031199B20B30B96280310851953
:100120000314B90DF03039020319562160238928D0
:1001300064003210080031110130B7008B132030F9
:10014000370783169B001C141A088312A400103072
:10015000370783169B001C141A088312A300A600FD
:100160000230A6060030370783169B001C141A08BD
:100170008312A200A7000130A7068B17321CC628E5
:1001800022090339A200A309A409A50924082F0202
:10019000031D502923082E02031D502922082D0279
:1001A000031D502901303702031DDB283D18DB28D1
:1001B0003D143E14072202303702031DE428BD1807
:1001C000E428BD143E14162203303702031DED2827
:1001D0003D19ED283D153E14222204303702031D3F
:1001E000F628BD19F628BD153E142E22053037021B
:1001F000031DFF283D1AFF283D163E143D22063000
:100200003702031D0829BD1A0829BD163E144C22C9
:1002100007303702031D11293D1B11293D173E14DC
:100220005B2208303702031D1A29BD1B1A29BD178E
:100230003E146A2209303702031D23295E18232940
:100240005E143E1475220A303702031D2C29DE1875
:100250002C29DE143E1480220B303702031D352971
:100260005E1935295E153E148B220C303702031DB2
:100270003E29DE193E29DE153E1496220D30370246
:10028000031D47295E1A47295E163E14A1220E302F
:100290003702031D5029DE1A5029DE163E14AC2207
:1002A000B70A0F303702031808009E280130B60045
:1002B000B300B400B500B70085018701B1139820E1
:1002C000B30BA629031085190314B90DF0303902B8
:1002D0000319CD29B40BA629013037020319B7221F
:1002E000023037020319BC22033037020319C1223E
:1002F000043037020319C622053037020319CB2216
:10030000063037020319D022073037020319D522ED
:10031000083037020319DA22093037020319DF22C5
:100320000A3037020319E4220B3037020319E9229D
:100330000C3037020319EE220D3037020319F32275
:100340000E3037020319F8229630B400311D5F29B0
:100350003111321CB0292D090339AD00AE09AF09A6
:100360002F1C5F298E018F010C1C5F290C102E1E83
:100370005F298B1320303707BB002F08BA00E52117
:1003800010303707BB002E08BA00E52100303707D0
:10039000BB002D08BA00E5218B1785018701B70A3C
:1003A000B6010F303702031C5F29FD2208003E1CF6
:1003B00008003E101030BB003D08BA00E521303087
:1003C000BB005E08BA00E52108008B133A088316CB
:1003D0001C159A0083123B0883169B0055309D0024
:1003E000AA309D009C1464009C18F3291C118312F0
:1003F0008B170800FF30C800CA15CB15CC15CD15DA
:10040000CE15CF15D015D115D215D31508008130D2
:10041000BD05FF30DE050130C405C0000030C2005C
:10042000C600BC185F14BC18DF1408008230BD057C
:10043000FF30DE050230C405C0000030C200C60037
:100440005F1008008430BD05FF30DE050630C405AE
:10045000C0000030C200C6005F1008008830BD0533
:10046000FF30DE050930C405C0000830C200C600F8
:10047000BC185F14BC18DF1408009030BD05FF30B5
:10048000DE051930C405C0000030C200C600BC182B
:100490005F14BC18DF140800A030BD05FF30DE0576
:1004A0002130C405C0000030C200C600BC185F1473
:1004B000BC18DF140800C030BD05FF30DE05103069
:1004C000C405C0000030C200C600BC185F14BC18D0
:1004D000DF140800FF30BD05C030DE055030C50513
:1004E000C1000030C300C70008007F30BD05C13027
:1004F000DE052030C505C1000030C300C70008007C
:100500007F30BD05C230DE05E030C505C1002030BA
:10051000C300C70008007F30BD05C430DE05503081
:10052000C505C1000030C300C70008007F30BD050D
:10053000C830DE055030C505C1000030C300C7001B
:1005400008007F30BD05D030DE055030C505C10044
:100550000030C300C70008007F30BD05E030DE0575
:100560004030C505C1000030C300C700080010308E
:100570008506003087060800203085060030870693
:1005800008002130850600308706080012308506F5
:100590000030870608001230850602308706080002
:1005A00010308506043087060800003085060230CA
:1005B00087060800003085061130870608000030E5
:1005C000850620308706080000308506383087060B
:1005D00008000030850611308706080000308506C7
:1005E00011308706080000308506113087060800A4
:1005F000003085063930870608003D180722BD18EF
:1006000016223D192222BD192E223D1A3D22BD1A65
:100610004C223D1B5B22BD1B6A225E187522DE1830
:1006200080225E198B22DE1996225E1AA122DE1A22
:10063000AC220800B601B301B4013C1C222BBC0162
:10064000BC14242BBC013C143C08B6006400282BCD
:10065000292B2A2B2B2B2C2BFF30B41B8500B41FEE
:100660008501B30B262BB40B262B0310B60CB60852
:10067000031D262B0030BB003C08BA00E521080012
:1006800005125C180516DC1C8512DC1885165C1D2D
:1006900005105C190514DC1D8510DC1985145C1E21
:1006A00087105C1A8714DC1E0711DC1A07155C1F03
:1006B00007105C1B0714DC1F8712DC1B8716080061
:1006C0008F08031908008F0178308E00C80F922D13
:1006D000C80A441C902B461C812BCA1C722BCA01D1
:1006E0004A159E2B4A1D772BCA01CA159E2BCA1D7F
:1006F0007C2BCA014A169E2B4A1E9E2BCA01CA1485
:100700009E2B4A1D862BCA014A169E2BCA1D8B2B77
:10071000CA014A169E2B4A1E9E2BCA01CA149E2B42
:10072000CA1C952BCA014A159E2B4A1D9A2BCA0139
:10073000CA159E2B4A1E9E2BCA014A15C41CC52BE6
:10074000C61CB62BCB1CA72BCB014B15D32B4B1D9B
:10075000AC2BCB01CB15D32BCB1DB12BCB014B1627
:10076000D32B4B1ED32BCB01CB14D32B4B1DBB2B2D
:10077000CB014B16D32BCB1DC02BCB014B16D32B50
:100780004B1ED32BCB01CB14D32BCB1CCA2BCB01B1
:100790004B15D32B4B1DCF2BCB01CB15D32B4B1E86
:1007A000D32BCB014B15441DFA2B461DEB2BCC1C38
:1007B000DC2BCC014C15082C4C1DE12BCC01CC15AD
:1007C000082CCC1DE62BCC014C16082C4C1E082CFA
:1007D000CC01CC14082C4C1DF02BCC014C16082C51
:1007E000CC1DF52BCC014C16082C4C1E082CCC0132
:1007F000CC14082CCC1CFF2BCC014C15082C4C1D08
:10080000042CCC01CC15082C4C1E082CCC014C150A
:10081000C41D302CC61D212CCD1C122CCD014D1514
:100820005F133E2C4D1D172CCD01CD153E2CCD1D3B
:100830001C2CCD014D163E2C4D1E3E2CCD01CD1451
:100840003E2C4D1D262CCD014D163E2CCD1D2B2CA6
:10085000CD014D163E2C4D1E3E2CCD01CD143E2C0F
:10086000CD1C352CCD014D153E2C4D1D3A2CCD0106
:10087000CD153E2C4D1E3E2CCD014D155F1B672C1A
:10088000441E672C461E582CCE1C492CCE014E15FA
:10089000752C4E1D4E2CCE01CE15752CCE1D532C15
:1008A000CE014E16752C4E1E752CCE01CE14752C15
:1008B0004E1D5D2CCE014E16752CCE1D622CCE0128
:1008C0004E16752C4E1E752CCE01CE14752CCE1CDA
:1008D0006C2CCE014E15752C4E1D712CCE01CE15F3
:1008E000752C4E1E752CCE014E15C41E9C2CC61E9A
:1008F0008D2CCF1C7E2CCF014F15AA2C4F1D832C85
:10090000CF01CF15AA2CCF1D882CCF014F16AA2CB2
:100910004F1EAA2CCF01CF14AA2C4F1D922CCF0111
:100920004F16AA2CCF1D972CCF014F16AA2C4F1E65
:10093000AA2CCF01CF14AA2CCF1CA12CCF014F156C
:10094000AA2C4F1DA62CCF01CF15AA2C4F1EAA2CC6
:10095000CF014F15DF18D32C451ED32C471EC42CB6
:10096000D01CB52CD0015015E12C501DBA2CD00153
:10097000D015E12CD01DBF2CD0015016E12C501EFB
:10098000E12CD001D014E12C501DC92CD0015016FF
:10099000E12CD01DCE2CD0015016E12C501EE12CA4
:1009A000D001D014E12CD01CD82CD0015015E12C52
:1009B000501DDD2CD001D015E12C501EE12CD001B2
:1009C0005015DF180A2DC51E0A2DC71EFB2CD11C81
:1009D000EC2CD1015115182D511DF12CD101D1153F
:1009E000182DD11DF62CD1015116182D511E182D80
:1009F000D101D114182D511D002DD1015116182DE2
:100A0000D11D052DD1015116182D511E182DD101C2
:100A1000D114182DD11C0F2DD1015115182D511D98
:100A2000142DD101D115182D511E182DD10151159C
:100A3000DF18422D451F422D471F332DD21C242D78
:100A4000D2015215DF13502D521D292DD201D2157E
:100A5000502DD21D2E2DD2015216502D521E502D2A
:100A6000D201D214502D521D382DD2015216502DC4
:100A7000D21D3D2DD2015216502D521E502DD201A5
:100A8000D214502DD21C472DD2015215502D521D7B
:100A90004C2DD201D215502D521E502DD20152157F
:100AA000DF187B2DDF1B7B2DC51F7B2DC71F6C2DFA
:100AB000D31C5D2DD3015315892D531D622DD301F8
:100AC000D315892DD31D672DD3015316892D531EA0
:100AD000892DD301D314892D531D712DD3015316A4
:100AE000892DD31D762DD3015316892D531E892DA3
:100AF000D301D314892DD31C802DD3015315892DF7
:100B0000531D852DD301D315892D531E892DD30156
:100B10005315D7214008C4004108C5005F18DF14F1
:100B20005F1CDF104808C9000C304A05031D051280
:100B30000C304B05031D85120C304C05031D0510B0
:100B40000C304D05031D85100C304E05031D87101C
:100B50000C304F05031D07110C305005031D071005
:100B60000C305105031D87120C305205031D07126E
:100B70000C305305031D871149080E020318EC2D94
:100B800012304A05031D051612304B05031D85164C
:100B900012304C05031D051412304D05031D85143C
:100BA00012304E05031D871412304F05031D071523
:100BB00012305005031D071412305105031D87160E
:100BC00012305205031D071612305305031D8715F9
:100BD000FF304802031908008F08031D0800982001
:100BE00049080E02031CEC2D18304A05031D05129E
:100BF00006304A05031D051618304B05031D8512E6
:100C000006304B05031D851618304C05031D0510D5
:100C100006304C05031D051418304D05031D8510C5
:100C200006304D05031D851418304E05031D871031
:100C300006304E05031D871418304F05031D07119C
:100C400006304F05031D071518305005031D07100A
:100C500006305005031D071418305105031D871277
:100C600006305105031D871618305205031D071263
:100C700006305205031D071618305305031D871152
:0A0C800006305305031D8715080018
:084000000700030003000900A2
:02400E00CC33B1
:10420000010078007A007C007E007B0079007F004E
:104210007D007A0078007E007C007D007F00FF003A
:104220000200F200F600FA00FE00F200F600FA00CA
:10423000FE00F200F600FA00FE00F200F600FF00B9
:10424000FF00050005000500050009000900090040
:1042500009000D000D000D000D0011001100FF0000
:104260000100FF00FF00FF00FF00FF00FF00FF0054
:10427000FF00FF00FF00FF00FF00FF00FF00FF0046
:10428000FF00FF00FF00FF00FF00FF00FF00FF0036
:10429000FF00FF00FF00FF00FF00FF00FF00FF0026
:1042A000FF00FF00FF00FF00FF00FF00FF00FF0016
:1042B000FF00FF00FF00FF00FF00FF00FF00FF0006
:1042C000FF00FF00FF00FF00FF00FF00FF00FF00F6
:1042D000FF00FF00FF00FF00FF00FF00FF00FF00E6
:1042E000FF00FF00FF00FF00FF00FF00FF00FF00D6
:1042F000FF00FF00FF00FF00FF00FF00FF00DD00E8
:00000001FF
